:0600000000308A00112807
:10000800FF00030883120313EB000408EC000A083E
:10001800ED007E08EE008A119F2C24308400033006
:10002800FE002630FF0022208000840A0408253ABA
:1000380003192628FF0A0319FE0A17287E088A00D2
:100048007F0882002530840036308A113C208A11CE
:10005800A8308400F0308A113C208A118317703050
:1000680084007E308A113C208A1183018A11442839
:1000780064008001840A04060319003404063D283C
:100088008B138A1557258A118A11F0228A118A152D
:10009800CB258A118A11B4228A118A158A258A11D8
:1000A8008316031386128312031386128B171730D5
:1000B8008A1109238A11BA003A08A70002308A1166
:1000C80009238A11BA003A08A60006308A110923C2
:1000D8008A11BA003A08A5008A15A5258A11831243
:1000E80003130030C9000030C8000130C700C23017
:1000F800C6008A157F268A1115308A1109238A11AC
:1001080083120313BA003A08A7000B308A11092397
:100118008A11BA003A08A60013308A1109238A11F5
:10012800BA003A08A5008A11FB258A11013A031D75
:100138009E289F28E7280F308A1109238A118312E5
:100148000313BA003A08A70014308A1109238A1148
:10015800BA003A08A60014308A1109238A11BA0095
:100168003A08A5008A15A5258A11831203130030C1
:10017800C9000030C8000030C7001E30C6008A150C
:100188007F268A118A15A5258A1183120313003048
:10019800C9000030C8000030C7001E30C6008A15EC
:1001A8007F268A118A15A5258A1183120313003028
:1001B800C9000030C8000730C700D030C6008A1513
:1001C8007F268A113A2A8A1127238A1179088312ED
:1001D8000313BA003A07A83EBB003B08F8000030FA
:1001E800AC000030AD000030B7000030B80003109C
:1001F800003003180130B9002C293908BA003A0731
:10020800A83E831384000008BB000130840700085F
:10021800BC003908BD003D07780784003B08800012
:10022800840A3C0880003908BA003A07A83E8400CE
:100238000008BB00013084070008BC003B08B70772
:100248000318B80A3C08B8070130BA003A08B907D9
:1002580079083902031C3129322901293808C901D2
:10026800C9073708C801C8078A1124278A11FC3032
:1002780083120313BA003A08FA052B08C5002A08A6
:10028800C4002908C3002808C2008A15A5278A11B6
:10029800831203134508C9004408C8004308C7006F
:1002A8004208C6008A157F268A1103108312031399
:1002B800003003180130B600831603132908F10132
:1002C800F1072808F001F0078A1542258A118312E0
:1002D80003135508AB005408AA005308A900520894
:1002E800A8000E2A8A1542258A11831203132808AA
:1002F8005202BA005308BB002908031C290FBB028D
:100308005408BC002A08031C2A0FBC025508BD006B
:100318002B08031C2B0FBD027008BE007108BF001C
:10032800C001C1013D084102031DA4293C08400247
:10033800031DA4293B083F02031DA4293A083E02D5
:100348000318A729A829D6293608BA003A07780732
:10035800831384000008F000840A0008F1008A155D
:1003680042258A11831203135508AB005408AA00CA
:100378005308A9005208A8000130BA003A08B60785
:1003880079083602031CC929CA29CF29031000306D
:1003980003180130B60086168A15A5258A1183121E
:1003A800031386127A0803390319DB29DC290E2A7C
:1003B8007A1CDF29E029E9297908BA00BB013A0843
:1003C800AC070318AD0A3B08AD07FA1CEC29ED2968
:1003D800F6297908BA00BB013A08AC023B08031CAD
:1003E800AD03AD02FC30BA003A08FA05062A7908CE
:1003F80083120313BA00BB013A08AC023B08031C82
:10040800AD03AD028A113D228A11013A03190D2A62
:100418000E2AFB298A15F3258A110030831203134B
:100428004702473003194602031C1B2A1C2A762957
:100438000030C9000030C8000030C700C830C6000E
:100448008A157F268A118A15A5258A118312031316
:100458000030C9000030C8000030C7001E30C60098
:100468008A157F268A118A15A5258A1180288A115E
:1004780011280030C2000030C300031000300318F8
:100488000130C400A22A4408C5004507A83E8313CA
:1004980084000008E100840A0008E2006030DF0000
:1004A800EA30E0008A15BA268A11831203132C0851
:1004B8005F07E1002D0803182D0A6007E20060308D
:1004C800DF00EA30E0008A15BA268A118312031386
:1004D8004408C60046077807831384005F08800035
:1004E800840A600880004408C5004507780784002E
:1004F8000008C600013084070008C7000030470222
:100508000A300319460203188A2A8B2A8D2A0130D9
:10051800B32A4408C5004507780784000008C600C8
:10052800013084070008C7004608C2070318C30A39
:100538004708C3070130C5004508C40779084402C5
:10054800031CA72AA82A472A4308C901C907420841
:10055800C801C8078A1124278A110030B32A080065
:10056800F83083120313C200831603138312031394
:100578004208831603138505F83083120313C2005B
:1005880042088505203083160313870017308A1127
:1005980009238A11831203138700031000300318FC
:1005A8000130F7000130C2004208FC0017308A1100
:1005B80009238A11C2004208A50017308A110923AD
:1005C8008A11C2004208A60017308A1109238A112D
:1005D800C2004208A70008008316031306178617EF
:0C05E800811383120317151795170800E4
:10060000FE00FE1F082B83137E18831700080800C6
:100610000408FE0003308A007E0882070034A034FC
:10062000F93464347034393432342234F8342034B8
:100630003034283423346734613426342E346B3418
:1006400063342C346F3427347734FF340A34F90898
:10065000031D2B2B2C2B252CFF3083120313CB00D7
:10066000FF30CC00F9010314F90D0330E100003034
:10067000E2000130D900DA0176085907DF005A0894
:1006800003185A0AE0008A15BA268A118312031346
:100690005F08013EC6000130CF000030D000182CAA
:1006A0000030C4000030C5000030D3000030D4005A
:1006B000DD2B5008E201E2074F08E101E107FF30BE
:1006C000D900FF30DA0076085907DF005A0803180E
:1006D0005A0AE0008A15BA268A11831203135F08AA
:1006E000FF3ED50060080318013EFF3ED6000030F3
:1006F000D7000030D800CD2B5008E201E2074F08A8
:10070000E101E1075808E001E0075708DF01DF07D2
:100710008A151D268A118312031353085F07C90027
:1007200054080318540A6007CA004F084907C70055
:1007300050080318500A4A07C8004708D90059074B
:10074000A83E831384000008DA0001308407000803
:10075000DB004908DC005C07A83E84000008DD00DF
:10076000013084070008DE005A085D02DF005B08E4
:10077000031C5B0A5E02E0008A152E258A11831293
:1007800003135F08C4070318C50A6008C5070130D2
:10079000D7070318D80A0030D80756085802031D97
:1007A000D32B55085702031CD62BD72B7C2B01309B
:1007B000D3070318D40A0030D40750085402031D8D
:1007C000E32B4F085302031CE62BE72B592B500851
:1007D000E201E2074F08E101E1074508E001E00717
:1007E0004408DF01DF078A151D268A1183120313CF
:1007F0006008C501C5075F08C401C4074C0845026D
:10080000031D042C4B0844020318072C082C122C3F
:100810004F08D9005908F9004508CC01CC07440815
:10082000CB01CB070130CF070318D00A0030D00727
:100830004608D900DA015A085002031D212C590834
:100840004F02031C242C252C502B790883120313F0
:10085000DF0076088A11CD278A1183120313D9008D
:10086000DA015908C2005A08C3000030CD00003038
:10087000CE00912C0030C4000030C5000030D10003
:100880000030D200652C5108DF0079088A157025E8
:100890008A1183120313D9004D085907DA005A0749
:1008A000A83E831384000008DB00013084070008A1
:1008B000DC005B08C4070318C50A5C08C5070130E3
:1008C000D1070318D20A0030D20743085202031D91
:1008D0006B2C42085102031C6E2C6F2C432C4308D6
:1008E000E201E2074208E101E1074508E001E00713
:1008F0004408DF01DF078A15BA268A118312031321
:100900004D08D9005907A83E831384005F08800072
:10091000840A600880000130CD070318CE0A003039
:10092000CE077908D900DA015A084E02031D9A2C25
:1009300059084D02031C9D2C9E2C3A2C08008B1E3E
:10094000A22CA32CF02D0B1DA62CA72CF02D0130D2
:10095000A4023A308100A408031DAF2CB02C922DC4
:100960000A30E7006708A4000130B2070030031125
:100970000318013E031DB307003003110318013EA5
:10098000031DB407003003110318013E031DB50712
:100990000330E7000030E8000030E9000030EA00F2
:1009A0003208E7053308E8053408E9053508EA05A3
:1009B0006A08690468046704031DDF2CE02C922D8B
:1009C0000310FD0D0310FB0D061FE72CE82CE92C8E
:1009D0007D14861FEC2CED2CEE2C7B14FD08031DE2
:1009E000F22CF32C352D7A1DF62CF72C052D7A14CC
:1009F000FB30E7006708FA053508F5003408F40015
:100A00003308F3003208F200352D72083202E70095
:100A10003308E8007308031C730FE8023408E90088
:100A20007408031C740FE9023508EA007508031CFA
:100A3000750FEA0200306A02031D282D003069029A
:100A4000031D282D00306802031D282D6530670224
:100A5000031C2B2D2C2D352D7A143508F500340868
:100A6000F4003308F3003208F2007D08FF3A031D5A
:100A70003A2D3B2D402D7A193E2D3F2D402D7A15D4
:100A8000FB08031D442D452D872DFA1D482D492DAA
:100A9000572DFA14F730E7006708FA053508B1005A
:100AA0003408B0003308AF003208AE00872D2E089E
:100AB0003202E7003308E8002F08031C2F0FE8027A
:100AC0003408E9003008031C300FE9023508EA0059
:100AD0003108031C310FEA0200306A02031D7A2D2F
:100AE00000306902031D7A2D00306802031D7A2D43
:100AF00065306702031C7D2D7E2D872DFA14350885
:100B0000B1003408B0003308AF003208AE007B08F3
:100B1000FF3A031D8C2D8D2D922DFA19902D912DBC
:100B2000922DFA150130FC02FC08031D982D992D19
:100B3000EF2D771D9C2D9D2DD12D0130E7006708ED
:100B4000FC000130E7006708F70777080339033A2C
:100B5000031DAB2DAC2DB02DFC30E7006708F70569
:100B60002030E7006708870577080339253E83139F
:100B700084000008E70067088704FB30E700670887
:100B8000F7050130E70077080339013EC92D03104E
:100B9000E70DFF3E031DC72D6708E80068088504C0
:100BA000EF2D0130E70077080339013ED92D0310FE
:100BB000E70DFF3E031DD72D6708FF3AE8006808E0
:100BC0008505F71DE42DE52DEA2D0330E7006708C4
:100BD000FC00EE2D2830E7006708FC0077150B11AC
:100BE0006E08FE006D088A006C0884006B088300A4
:100BF000FF0E7F0E0900FE30C2004208F900002EF1
:100C00008A15F3258A1100308312031347024730F7
:100C100003194602031C0D2E0E2E002E7908FE3AF3
:100C2000031D132E142E192E03100030031801304B
:100C3000F90015308A1109238A11C2004208A70061
:100C40000B308A1109238A11C2004208A600133012
:100C50008A1109238A11C2004208A5008A1542257B
:100C60008A11831203135508AB005408AA005308D5
:100C7000A9005208A800F7150030C9000030C800CC
:100C80000030C7001E30C6008A157F268A11F73053
:100C900083120313C2004208F7054E2E8A15F3256E
:100CA0008A110030831203134702473003194602AA
:100CB000031C5B2E5C2E4E2E8A1542258A11831250
:100CC00003132808520283160313A8008312031388
:100CD0002908031C290A530283160313A9008A1545
:100CE00042258A11831203135508AB005408AA0049
:100CF0005308A9005208A800F7150030C9000030B9
:100D0000C8000030C7001E30C6008A157F268A1131
:100D1000F73083120313C2004208F705F6010314EB
:100D2000F60DFC30C2004208FA05DF2E8A15F325C5
:100D30008A1100308312031347024630031946021A
:100D4000031CA32EA42EDF2E8A1542258A1183129E
:100D5000031328085202C2002908031C290A53025F
:100D6000C3007608C4004407A83E831384004208E9
:100D70008000840A430880008A1542258A11831264
:100D800003135508AB005408AA005308A9005208E1
:100D9000A800F7150030C9000030C8000030C700B7
:100DA0001E30C6008A157F268A11F730831203137E
:100DB000C2004208F7050130C2004208F6078A1552
:100DC00042258A118312031328085202C2005308D5
:100DD000C3002908031C290FC3025408C4002A08B1
:100DE000031C2A0FC4025508C5002B08031C2B0F37
:100DF000C50200304502031D072F00304402031DC9
:100E0000072F07304302031D072FD030420203187B
:100E10000A2F0B2F192F243076020318102F112FB1
:100E2000192F7A18142F152F192FFA1C182F192F74
:100E3000962E7608243A031D1E2F1F2F212F0130D6
:100E4000232F0030232F08004908E201E207480859
:100E5000E101E1076030DF00EA30E0008A15BA26E0
:100E60008A11831203136008CB01CB075F08CA0104
:100E7000CA070A30CF000030D0004B08CE01CE07A1
:100E80004A08CD01CD078A1547268A11831203131C
:100E90004D08013E8A1109238A11CC004C08A50097
:100EA0000A30E1000030E2004B08E001E0074A08A8
:100EB000DF01DF078A15BA268A118312031360083F
:100EC000CB01CB075F08CA01CA070A30CF00003048
:100ED000D0004B08CE01CE074A08CD01CD078A15B8
:100EE00047268A11831203134D08013E8A110923F4
:100EF0008A11CC004C08A6000A30E1000030E20064
:100F00004B08E001E0074A08DF01DF078A15BA262F
:100F10008A11831203136008CB01CB075F08CA0153
:100F2000CA070A30CF000030D0004B08CE01CE07F0
:100F30004A08CD01CD078A1547268A11831203136B
:100F40004D08013E8A1109238A11CC004C08A700E4
:100F500001308A1109238A11CC0027084C06031D91
:100F6000B22FB32FCC2F17308A1109238A11CC004E
:100F70004C08A70001308A1109238A11CC002608E9
:100F80004C06031DC42FC52FCC2F17308A110923FF
:100F90008A11CC004C08A6000800E00003100030C5
:100FA00003180130E200DF08031DD72FF82FE101FD
:100FB0000314E10DE12F0310DF0D0130E30063089E
:100FC000E107DF1FE42FE52FDB2F0310E20D5F08A1
:100FD0006002031CEC2FED2FF02F5F08E00262147B
:100FE0000310DF0C0130E102031DF72FF82FE52F6E
:060FF0006208FA2F080060
:101A5C00E01F312D322D402D6008E2005F08E100BF
:101A6C00E109E209E10A0319E20A6108DF006208F0
:101A7C00E000412D412D080083128B133508D9004D
:101A8C003408D8003308D7003208D6008B17590811
:101A9C00D5005808D4005708D3005608D200562D4C
:101AAC000800831603130616031083120317003065
:101ABC00031801309E0003100030031801309F0002
:101ACC001F155030831603139F00A9308312031384
:101ADC009F000800E0000310003003180130E10003
:101AEC00601C792D7A2D7E2D5F08E2006208E107DB
:101AFC000310DF0D0310E00CE008031D862D872D6D
:101B0C00762D6108892D08008316031381153A3050
:101B1C008312031381008B168B170B1103100030EB
:101B2C0003180130A4000030B5000030B4000030C0
:101B3C00B3000030B2008316031381120800831621
:101B4C0003138712F715831203130030C9000030FA
:101B5C00C8000030C7001430C6008A157F268A15CD
:101B6C00831603138716F73083120313C20042083F
:101B7C00F7050030C9000030C8000030C700013044
:101B8C00C6008A157F268A1508008316031387164C
:101B9C000C30831203139700861BD52DD62DDB2D0D
:101BAC009C30831603139200E82D061BDE2DDF2DCF
:101BBC00E42D6830831603139200E82D7C308316D5
:101BCC0003139200120883120313C2000310420C79
:101BDC0095008C100530920008008312031303301B
:101BEC00C800C80BF72D831203139F14FD2D9F18EB
:101BFC00002E012EFD2D83160313831203131E08D2
:101C0C00C800C9010830CA000310C80DC90DCA0BA1
:101C1C000A2E831603131E08831203134807C600EB
:101C2C000030031801304907C7001C2E0800003093
:101C3C00E3000030E4005F1C242E252E2B2E6108BF
:101C4C00E3070318E40A6208E40701300310E10D0E
:101C5C00E20DFF3E031D2C2E01300310E00CDF0CB7
:101C6C00FF3E031D332E60085F04031D3E2E3F2EE6
:101C7C00212E6408E001E0076308DF01DF07462E30
:101C8C00080050084F0403194C2E4D2E7D2ED10107
:101C9C000314D10D5C2E01300310CF0DD00DFF3E7F
:101CAC00031D522E0130D2005208D107D01F5F2ED7
:101CBC00602E512E50084E02031D662E4F084D0209
:101CCC00031C692E6A2E702E4F08CD025008031C7F
:101CDC00CE03CE0201300310D00CCF0CFF3E031DFF
:101CEC00712E0130D102031D7C2E7D2E602E7E2E96
:101CFC0008008A1542258A15831203135508CD0056
:101D0C005408CC005308CB005208CA008D2E8A15FB
:101D1C0042258A15831203134A085202CE00530837
:101D2C00CF004B08031C4B0FCF025408D0004C08BB
:101D3C00031C4C0FD0025508D1004D08031C4D0F4D
:101D4C00D10251084902031DB52E50084802031D4B
:101D5C00B52E4F084702031DB52E4E084602031838
:101D6C00B82EB92E8D2E08000030E4000030E500AE
:101D7C00620861040319C32EC42EFF2EE301031461
:101D8C00E30DD32E01300310E10DE20DFF3E031DD8
:101D9C00C92E0130E6006608E307E21FD62ED72EC7
:101DAC00C82E01300310E40DE50DFF3E031DD82EA7
:101DBC0062086002031DE42E61085F02031CE72E1B
:101DCC00E82EF22E6108DF026208031CE003E00239
:101DDC000130E4040030E50401300310E20CE10CA6
:101DEC00FF3E031DF32E0130E302031DFE2EFF2EDA
:101DFC00D72E6508E001E0076408DF01DF07062F36
:101E0C000800590858045704560403190E2F0F2FB5
:101E1C00532FDA010314DA0D202F0130DB000310ED
:101E2C00D60DD70DD80DD90DDB0B152F0130DB00DE
:101E3C005B08DA07D91F232F242F132F59085502BB
:101E4C00031D322F58085402031D322F570853021A
:101E5C00031D322F56085202031C352F362F442FE8
:101E6C005608D2025708031C570FD3025808031CFC
:101E7C00580FD4025908031C590FD5020130031016
:101E8C00D90CD80CD70CD60CFF3E031D452F0130B6
:101E9C00DA02031D522F532F242F542F0800003029
:101EAC00D9000030D8000030D7000030D600003008
:101EBC00DA000030DB008E2F5A08DC005C07A83EED
:101ECC00831384000008DD00013084070008DE0065
:101EDC005D08DF005E08E000E101E2015F08D60763
:101EEC00600803110318600A031DD707610803116A
:101EFC000318610A031DD807620803110318620A4C
:101F0C00031DD9070130DA070318DB0A0030DB07A1
:101F1C007908DC00DD015D085B02031D972F5C086E
:101F2C005A02031C9A2F9B2F622F5908D500580870
:101F3C00D4005708D3005608D200A42F08008A15E5
:101F4C0055278A15831203135508C9005408C80075
:101F5C005308C7005208C6008A1542258A158312F9
:101F6C00031342085202CA005308CB004308031C57
:101F7C00430FCB025408CC004408031C440FCC0282
:101F8C005508CD004508031C450FCD024D08D50062
:101F9C004C08D4004B08D3004A08D2004908D90099
:101FAC004808D8004708D7004608D6008A150727E6
:101FBC008A158312031352084602CE004708CF003D
:101FCC005308031C530FCF024808D0005408031CBD
:101FDC00540FD0024908D1005508031C550FD102EB
:101FEC005108C5005008C4004F08C3004E08C20079
:041FFC00FF2F0800AB
:02400E00E2309E
:00000001FF
